:100000000C943B030C9458030C9458030C94580321
:100010000C9458030C9458030C9458030C945803F4
:100020000C9458030C9458030C94F7120C94391246
:100030000C94231B0C9458030C9458030C945803F1
:100040000C9458030C9458030C9458030C945803C4
:100050000C94ED1D0C9479140C9458030C945803D3
:100060000C9458030C9458030C9458030C945803A4
:100070000C9458030C9458030C9458030C94580394
:100080000C9458030C9458030C9458030C94580384
:100090000C9458030C9458030C9458030C94580374
:1000A0000C9458030C9458030C9458038105830551
:1000B000DC058B05C3059B05E9054C06C006540607
:1000C0001E062206580625065B0666063006B6069C
:1000D00034066A0638066E0698063C067206A206C4
:1000E00042067806820629065F062C066206470647
:1000F0007D068E06AE06B0061A065006C906EF0645
:10010000F506E306E906FB0601070707B607B6078B
:10011000E807E80767088308840984098808FC0859
:100120000D090D093D0D400D7B0D940D9B0DA60D88
:10013000A90DA90DA90D870E870EED0DEF0DF40D7C
:100140001A0E3C0E3F0E420E660E51107810211210
:1001500078102112C410E7102112DC11EC110000FC
:10016000000000000000000000000000000000008F
:10017000000000000000000000000000000000007F
:1001800000007E0F00D4FFFFFFC7000000780000D2
:100190000000000000002A2B2800000000000000E2
:1001A00000000000000000000029000000002C1EDC
:1001B0003420212224342627252E362D3738271E99
:1001C0001F202122232425263333362E37381F04BF
:1001D00005060708090A0B0C0D0E0F101112131457
:1001E00015161718191A1B1C1D2F3130232D350415
:1001F00005060708090A0B0C0D0E0F101112131437
:1002000015161718191A1B1C1D2F3130354C0501F6
:100210000902A10185020901A100050919012908A6
:100220001500250195087501810205010930093184
:100230001581257F95027508810609381581257F6E
:10024000950175088106050C0A38021581257F95F0
:100250000175088106C0C005010980A10185031947
:10026000012AB700150126B700950175108100C05D
:10027000050C0901A101850419012AA00215012616
:10028000A002950175108100C005010906A1018534
:1002900006050719E029E715002501950875018174
:1002A000020507190029EF1500250195F075018158
:1002B0000205081901290595057501910295017539
:1002C000039101C00660FF0961A1010962150026C2
:1002D000FF009520750881020963150026FF00952F
:1002E0002075089102C005010906A101050719E062
:1002F00029E715002501950875018102950175080A
:1003000081010507190029FF150026FF00950675D4
:1003100008810005081901290515002501950575B5
:10032000019102950175039101C009025B0003016F
:1003300000A0FA09040000010301010009211101D4
:10034000000122440007058103080001090401009F
:10035000020300000009211101000122220007050B
:1003600082032000010705030320000109040200A5
:10037000010300000009211101000122B600070558
:1003800084032000011201000200000008254068DB
:100390004D0101010200010A034D004600360038FC
:1003A0000000000C03640069003000690062000076
:1003B0000004030904000000000000000000000029
:1003C00001010203040506080A0C0F1114181C2071
:1003D00024292E33393F464C535B626A7179818AF6
:1003E000929AA2AAB2B9C1C8CFD5DCE1E7EBF0F48A
:1003F000F7FAFCFDFEFFFEFDFCFAF7F4F0EBE7E197
:10040000DCD5CFC8C1B9B2AAA29A928A8179716AA1
:10041000625B534C463F39332E2924201C1814119B
:100420000F0C0A0806050403020101000000000089
:10043000000000000029001E001F002000210022F3
:1004400000230024002500260027002D002E002A6E
:100450000049004B002B0014001A0008001500177B
:10046000001C0018000C00120013002F0030003197
:10047000004C004E00390004001600070009000A75
:10048000000B000D000E000F00330034002800E1C7
:10049000001D001B000600190005001100100036A9
:1004A0000037003800E5005200E000E300E2002CD5
:1004B000002152E600E400500051004F000000000F
:1004C000000000000035003A003B003C003D003ECB
:1004D000003F004000410042004300440045002A24
:1004E00000A9004A000100010001005200010001C2
:1004F0000001000100010001000100010005780178
:1005000000AA004D0001000100500051004F000101
:1005100000010001000100010001000100010001D3
:1005200000010001000100010001000100A800011C
:1005300000010001000100A800010001000100010C
:1005400000010001000100AC00AE00AB00000000A3
:100550000000000000010001000100010001000195
:100560000001000100010001000100010001000183
:100570000001000100010001000100010001000173
:100580000001000100010001000100010001000163
:100590000001000100010001000100010001000153
:1005A0000001000100010001000100010001000143
:1005B0000001000100010001000100010001000133
:1005C0000001000100010001000100010001000123
:1005D0000001000100010001000100010000000015
:1005E0000000000000010001000100010001000105
:1005F00000010001000100010001000100010001F3
:1006000000010001000100010001000100010001E2
:1006100000010001000100010001000100010001D2
:1006200000010001000100010001000100010001C2
:1006300000010001000100010001000100010001B2
:1006400000010001000100010001000100010001A2
:100650000001000100010001000100010001000192
:100660000001000100010001000100010000000084
:1006700000000000000011241FBECFEFDAE0DEBF53
:10068000CDBF11E0A0E0B1E0EEEFF6E402C00590CE
:100690000D92A636B107D9F722E0A6E6B1E001C077
:1006A0001D92AB38B207E1F70E94FB090C947D2341
:1006B0000C940000A6E0B0E0E0E6F3E00C944823E0
:1006C00049835A8349815A81992361F0222351F049
:1006D000CA010E94281F182F682F89819A810E94C1
:1006E000981F04C0CA010E94641F182F69817A8173
:1006F000812F0E94C3162696E3E00C9464230E9487
:100700000F202FEF84E39CE0215080409040E1F7E0
:1007100000C000009AE088E10FB6F894A895809395
:1007200060000FBE90936000FFCFABE1B0E0EBE95B
:10073000F3E00C9447234E8B5F8B688F798F8A8F01
:100740009B8F192F91111092FC01DE011F9687E0FB
:10075000FD0111928A95E9F786E0FE0176960190F7
:100760000D928A95E1F70A8D002341F021E04F8533
:10077000588969897A89C8010E945A030B8B1C8B9E
:1007800087E0FE013F96DE01189601900D928A9552
:10079000E1F7CE0108960E94FC1881112CC087E079
:1007A000FE013896DE01119601900D928A95E1F7CF
:1007B0006C85662301F12091C00130E0C9010196EA
:1007C000877099274091F90150E08417950761F1EE
:1007D0006D8397E0929FD001939FB00D1124AF538A
:1007E000BE4FFE01319601900D929A95E1F78093EC
:1007F000C0010E94991817E08091F9019091C00101
:100800008917F9F0189FC00111248F539E4F0E9441
:10081000FC188823B1F08091F90190E0019687706F
:1008200099278093F901E8CF0E940F201092C00110
:100830001092F901E9EBF1E087E0DF011D928A9562
:10084000E9F76B96E4E00C946323A8E0B0E0EBE2F8
:10085000F4E00C943923FC018481882309F4C7C592
:100860007F0121E0408151816281738195810E94E5
:100870005A038C01F7018581882309F4B4C19801DA
:1008800037572038310508F032C1003108F0DBC29B
:100890008FEF93E00E9466228111D5C238E6A32E25
:1008A00032E0B32E002379F0A114F4E0BF0609F47E
:1008B000CAC2C5010E946622811101C001502FEFFA
:1008C000A21AB20AEFCFCE0101962C0188E0F20104
:1008D00011928A95E9F72AE0322E85010F5F1F4FAA
:1008E000C5010E94662289831A82882309F4ABC25B
:1008F000813009F041C06501F2E0CF0ED11CC80182
:100900000E9466228A83882309F49DC29FEF980F74
:10091000933060F423E0A20EB11CC6010E9466224F
:100920008B83882309F48FC21C8229C0843031F55F
:100930004E0133E0830E911C02E010E056018FEF70
:10094000A81AB80AC6010E946622F40181934F01D9
:10095000882309F478C28C3741F4E2E0F0E0EC0F30
:10096000FD1FE00FF11F10820AC00F5F1F4F6501CE
:100970000730110519F767C2580101C056018201FD
:10098000F8012081222309F4A8CF213009F053C0B7
:100990008181813081F46801F2E0CF0ED11CF80131
:1009A0008281893319F460E570E002C060E070E094
:1009B0000E944E2215C0823049F46801F2E0CF0E49
:1009C000D11CF80182810E9497210AC0833051F422
:1009D0006801F2E0CF0ED11CF80182810E943D2116
:1009E000860182C0843019F00F5F1F4F7DC0F8016F
:1009F00022810E5F1F4F80E090E030E020533109EC
:100A00002A30310568F4389EA001399E500D11241A
:100A1000C901840F951F0F5F1F4FF8012081EDCF93
:100A2000009709F461C0EFE9FFE03197F1F700C0EA
:100A300000000197F5CFE22FF0E0E257FE4F24903F
:100A4000822F86958695869590E0FC01E258FE4FB0
:100A500064902770712C022E02C0759467940A94DA
:100A6000E2F7F1E06F227724FC01E259FE4F849017
:100A7000912C022E02C0959487940A94E2F731E0FB
:100A800083229924FC01E25AFE4FC490D12C02C06B
:100A9000D594C7942A95E2F781E0C822DD24611439
:100AA000710419F081EE0E9497218114910419F0CC
:100AB00086EE0E94972160E070E0822D0E944E2217
:100AC0008114910419F086EE0E943D216114710495
:100AD00019F081EE0E943D21C114D10429F060E09B
:100AE00070E08CE20E944E220F5F1F4F49CFF80149
:100AF000F857E730F10508F076C0EA5AFF4F0C943A
:100B0000122383E001C080E00E94C21E8091530244
:100B10000E94911E98C180915302982F96959695A8
:100B2000969549F1915E990F990F990F8770892BCE
:100B30008093530214C090915302892F8695869515
:100B400086958F5F8F719770843008F03FC0880F53
:100B5000880F880F892B8093530280915302887FDE
:100B600091E009F490E08091530290FB80F980932A
:100B700053020E94911E8091530286958695869518
:100B80000E94661E60C120915302822F8695869531
:100B90008695482F50E04330510554F48F5F982FCD
:100BA000990F990F990F822F8770892B8093530289
:100BB000809153028160DBCF8091530280FF03C09C
:100BC0000E94DC1E40C10E94E91E3DC19093530269
:100BD000C4CF8091530281FF03C00E94971E33C18E
:100BE0000E94AD1E30C1F801E851FC47E730F10525
:100BF00008F4E5C0882309F43AC110926602C801DE
:100C00009057839708F00CC184E090E00E946E2218
:100C100090936E0280936D02F801E150F047E2324A
:100C2000F10520F4E35AFF4F0C94122380916D02DA
:100C30008160ACC080916E028860B4C080916D020A
:100C40008260A4C080916D0220C080916D02886096
:100C50009DC080916E021EC080916E028260A2C013
:100C600080916D02806192C080916D0280628EC021
:100C700080916D0280648AC00E940F2080916D0275
:100C8000806884C080916D02886084607FC080919C
:100C90006E028260816086C080916D028E7F76C018
:100CA00080916E02877F7EC080916D028D7F6EC0C5
:100CB00080916D0220C080916D02877F67C0809116
:100CC0006E021EC080916E028D7F6CC080916D029D
:100CD0008F7E5CC080916D028F7D58C080916D02C7
:100CE0008F7B54C00E940F2080916D028F774EC081
:100CF00080916D02877F8B7F49C080916E028D7FCE
:100D00008E7F50C080916D0282FB222720F991E0F6
:100D1000922790FB82F990FB83F938C080916E0294
:100D2000982F909591708E7F892B90FB81F93AC016
:100D300080916D0286FB222720F991E0922790FB9B
:100D400086F924C00E940F2080916D0287FB222724
:100D500020F991E0922790FB87F918C061E001C06B
:100D600060E08EE090E00E9484221EC080916D02BF
:100D700084FB222720F991E0922790FB84F906C09A
:100D800080916D02982F909590FB80F980936D0271
:100D90000BC080916E0283FB222720F991E09227FD
:100DA00090FB83F980936E0260916D0270916E02E8
:100DB00084E090E00E94A2220E940F2044C0E158EB
:100DC000FF4F0C94122306E221EE41EE6AE17CE72C
:100DD00023C007E225EE45EE6BE17CE71DC006E28D
:100DE00021EE40EE68E17CE717C007E225EE44EE15
:100DF00069E17CE711C006E221EE42EE6CE17CE79E
:100E00000BC007E225EE46EE6DE17CE705C008E287
:100E100021E045EE6EE17CE7C7010E94451C13C04E
:100E20000631FCE71F0799F5809125028A7A91E047
:100E300009F490E090936801811117C089E20E9443
:100E40007A1B0E9419188091FA01877009F4CFC2A9
:100E5000F7018581882309F4CAC280916E0282FF5E
:100E6000C6C282E00E946B18C2C285E3E8CF063199
:100E70002CE7120709F470C20737FCE71F0709F4D3
:100E8000A5C208372CE7120709F4A8C21AC0073711
:100E90003CE7130709F49CC208378CE7180709F4EC
:100EA00099C203309CE7190709F47CC208F05EC2BE
:100EB0000115FCE71F0709F467C201301C4709F45C
:100EC00077C2F701858100811181882349F0C8012B
:100ED0000E94281FD82E682FC8010E94981F04C0A6
:100EE000C8010E94641FD82EB8018D2D0E94C31620
:100EF0000E94D1168C01A82EF701B580968092949D
:100F00009FE099228091FA01877001F1BB20F1F0F6
:100F1000812F807F803469F080E2800F8830B0F0CC
:100F2000812F807E803229F4F1E0F01778F4992047
:100F300069F080916E0282FF09C082E00E946B1806
:100F40008091FA018770DD24D3948111D12CC12EB8
:100F5000C2948FE0C8228C2D90E08C30910508F06F
:100F6000D3C1FC01EA57FF4F0C941223812F807FDD
:100F70001F70882311F01295107FBB20B9F0112348
:100F800009F4B0C180E2800F883010F0A11006C0D3
:100F900090912502192B1093250205C09091FC0118
:100FA000192B1093FC010E9419189CC1802F0E94DC
:100FB0003D21112309F4A8C1005E083080F1AA2068
:100FC00071F110959091FC0119231093FC012AC036
:100FD000812F807F1F70803211F01295107FAA2020
:100FE00029F021E0A21609F44DC058C080916E028C
:100FF00082FD1BC0BB2069F0112339F0309125021E
:10100000312B309325020E94191880E00E9497210D
:101010007BC180E00E943D21112309F475C1812F1D
:101020000E9412180E9419186FC1BB2081F09920EC
:10103000C9F131E0931268C13091FB01812F832304
:10104000181709F461C1312B3093FB015DC1911078
:101050005BC1812F0E9440203091FB01812F8323AF
:1010600029F0812F809538233093FB01209169016D
:10107000812F822309F448C1312F309523232093F7
:10108000690142C1BB2029F085E0891508F43CC103
:1010900009C094E0991508F437C115C0BB2031F0A0
:1010A000911020C1812F0E9447202EC1992059F014
:1010B000093309F026C1EFEFF7EE23E0E150F040ED
:1010C0002040E1F71CC1812F0E9440201DC1812FCB
:1010D00086958695837019F0813059F015C1BB2033
:1010E00019F0C801937002C080E090E00E94D61B06
:1010F00011C1BB2019F0C801937002C080E090E0DC
:101100000E94B11B07C16B2D802F0E94512002C18C
:10111000812F8370A9F5B110FBC0402F42954695F1
:101120004770440F440F802F8F7090E09C01042E75
:1011300001C0220F0A94EAF704FF08C08FE090E094
:1011400001C0880F4A95EAF7809501C080E01695A6
:1011500016951370123069F088F490917A0111306D
:1011600019F0822B892302C0922B892B0E94E91F40
:10117000CFC0822B90917A018927F8CF822BF6CFAE
:10118000BB2019F0812F817001C08695882309F456
:10119000BFC0402F429546954770440F440F802FA3
:1011A0008F7090E09C01042E01C0220F0A94EAF790
:1011B00004FF08C08FE090E001C0880F4A95EAF76D
:1011C000809501C080E0169516951370123059F085
:1011D00078F490917B01113019F0822B892309C09A
:1011E000922B892B06C0822B90917B01892701C00D
:1011F000822B0E94CD1F8CC01F70BB2039F0812F25
:101200000E94DD1F802F0E94472082C0802F0E94F5
:101210004020812F0E94D01F7BC0802F32EFA31669
:1012200081F13A1538F090EFA91659F0E1EFAE16BA
:1012300019F154C0F3EFAF1659F124EFA216C1F023
:101240004DC0BB2081F034E0391508F45DC01F713A
:1012500081E090E0012E01C0880F0A94EAF7909196
:101260007B01892720C085E0891508F44DC0EFCFA8
:1012700080916E0282FD1AC0BB2029F0812F8F71F0
:1012800020C0BB20D9F3812F8F710E94D01F3CC09A
:10129000BB2041F01F7181E0012E01C0880F0A942C
:1012A000EAF701C080E00E94CD1F2EC0BB2061F094
:1012B000812F8F7198E0899F9001112423602093E2
:1012C000FA010E94DD1F20C081E00E946B18E1E05E
:1012D000E915D0F482E00E946B1816C0BB2021F003
:1012E000992061F2802F92CE992069F2893349F4D6
:1012F000FFEF27EE33E0F15020403040E1F700C02F
:101300000000802F0E943D2188EF8C0D843010F466
:101310000E94FB1BDD20A9F08091FA0180FD11C025
:10132000F70115828695869586950E94DD1FC70177
:101330000E9425048091FA018695869586950E94E3
:10134000D01F20E0F7014081518162817381848147
:1013500095810E945A034BC080916801811104C09D
:1013600089E20E944C1B6DCD85E3FBCF0B353CE73A
:10137000130741F10C358CE71807E1F00A351C47DB
:1013800009F09FCD81E01FC00E940F20EFEFF4E332
:101390002CE0E150F0402040E1F700C000000E9446
:1013A000681451CD6FEF7FEF80E090E00E94A222A1
:1013B0000E947F0380916E0282FB882780F991E072
:1013C000892701C080E00E9482187BCD81E007C0A0
:1013D00081E001C082E00E94DD1F03C082E00E9424
:1013E000D01F43E062E081E00E94831A2CCD289652
:1013F000E2E10C945523A6E2B0E0E1E0FAE00C94BF
:10140000392385B7806885BF85B7806885BF84B775
:10141000877F84BF0FB6F894A8958091600088619B
:1014200080936000109260000FBE90E080E80FB6DD
:10143000F89480936100909361000FBE86EC94E174
:1014400090936701809366010E947D120E949C1216
:101450008091E20084608093E20078948091AF01F3
:101460008823A1F01091E9001F709091EC00892F62
:10147000817090FD80E8182B1092E9008091E800BF
:1014800083FD0E946E0F1F701093E90082E084BDFF
:1014900093E095BD9AEF97BD80936E000E942C1C3F
:1014A000811102C00E94AF1D0CE011E0D8018D91A6
:1014B0008D018F3F11F00E94F915B1E004311B0737
:1014C000A9F704E111E0F80181918F018F3F11F03C
:1014D0000E94F915F1E00D311F07A9F780E1EEE850
:1014E000F1E0DF01282F1D922A95E9F7EAE6F1E005
:1014F000DF011D928A95E9F780E090E00E946E225C
:10150000853E9E4F21F40E942C1C811163C065EE24
:101510007EEF80E090E00E94A22260E082E090E016
:101520000E94842281E080937A0161E083E090E070
:101530000E94842260E074E184E090E00E94A22294
:1015400060E086E090E00E94842260E087E090E026
:101550000E94842240E050E0BA0188E090E00E94BE
:10156000962260E083E290E00E94842260E08CE0BA
:1015700090E00E94842260E08DE090E00E9484224E
:1015800019821A821B821C821D821E821F8218866B
:1015900048E050E067E170E0CE0101960E947422BD
:1015A00040E050E0BA018FE190E00E94962280E096
:1015B0000E940D1C0E94AF1D40E050E0BA018FE078
:1015C00090E00E94962240E050E0BA0183E190E072
:1015D0000E94962282E090E00E94662280937C0125
:1015E00084E090E00E946E2290936E0280936D02E0
:1015F0000E941016EFEFF6E721E0E150F0402040A6
:10160000E1F700C000000E94101680918E0180FF5B
:1016100008C06FEF7FEF80E090E00E94A2220E945E
:10162000681483E090E00E9466220E94E91F259AD8
:101630002D9882E88093800089E1809381008FEF6C
:101640009FEF90938700809386000E94011F8091F6
:10165000530281FF0BC01092560210925502109255
:10166000540280916F00816080936F000E94011F7F
:1016700080E091E090936A02809369029EE9492E8E
:1016800091E0592E8E010F5F1F4F8091AF01853081
:1016900009F04CC0B0E1EB2E82E1F82E8091AF0151
:1016A000853009F03DC08091AF01843039F180E090
:1016B0000E94C21E10926F0288E190E0A0E40FB673
:1016C000F894A895809360000FBEA093600083B744
:1016D000817F846083BF83B7816083BF789488955E
:1016E00083B78E7F83BF0FB6F894A8958091600072
:1016F000886180936000109260000FBE8091AE01FF
:10170000882309F4CBCF0E941016EEE8F1E0819116
:101710009191892B09F004C34E165F06C1F7BECF25
:101720000E940F200E94011F0E94FB1B0E941016A6
:10173000FDE7EF2EF1E0FF2EAEE86A2EA1E07A2E53
:10174000D301F701219131918D919D9182279327AA
:1017500021E0ED38F20719F0892BA1F305C0892BA0
:1017600019F40E94EE173FC0312CD3018D909D904B
:101770003D01F701A080B180A824B924A114B104CF
:1017800049F1212CCC24C394D12CC6018A219B2160
:10179000892BB9F029A23AA20E94BA149CA38BA368
:1017A000F1E0FDA391E0960128213921232B09F4D2
:1017B00090E09EA349A15AA16BA17CA18DA10E949A
:1017C00095032394CC0CDD1C29E02212DECFD70137
:1017D0008D929C923394B2E0EB0EF11CE8E03E1245
:1017E000C4CF0E94AE1486E0EEE5F2E0D80101908D
:1017F0000D928A95E1F7B0905F02D0906002F09070
:101800006102E0906202C090630210926002109246
:1018100061021092620210926302D11003C0FF2095
:1018200009F447C080915C0290915D020E949F1470
:101830009C0190915702992309F491C225313105F9
:10184000C0F19F3F19F09F5F90935702DD2061F038
:101850000E94151D1D1414F491E001C09FEF899F93
:10186000802D112480936002FF2061F00E94151DDD
:101870001F1414F09FEF01C091E0899F802D112467
:101880008093610280916002882399F0A0906102A8
:10189000AA2079F00E94351D811101C081E080935A
:1018A00060028A2D0E94351D811101C081E0809364
:1018B0006102E11003C0CC2009F447C080915A02B4
:1018C00090915B020E949F149C0190915802992371
:1018D00009F44AC221353105C0F19F3F19F09F5FDD
:1018E00090935802EE2061F00E94F31C1E1414F431
:1018F00091E001C09FEF899F802D112480936202A7
:10190000CC2061F00E94F31C1C1414F09FEF01C066
:1019100091E0899F802D112480936302809162025F
:10192000882399F0A0906302AA2079F00E94351DC7
:10193000811101C081E0809362028A2D0E94351DD1
:10194000811101C081E08093630280915F028B115D
:101950001AC080916002882311F08D1114C080910B
:101960006102882311F0F8120EC08091630288236F
:1019700011F08C1108C090916202992331F081E03E
:10198000E91204C002C081E001C080E080FD15C002
:101990008091600281110FC08091610281110BC0A2
:1019A00080916202811107C081E0909163029111E0
:1019B00003C080E001C081E080FD0E94C91CBA82A2
:1019C000DB82FC82ED82CE8286E0F801AEE5B2E0F9
:1019D00001900D928A95E1F70E94FB1B90918D0179
:1019E000891721F080938D010E94AE148091AF0180
:1019F000843009F04ACE83E08093E9008091E800CA
:101A000082FF43CE8091E80085FF21C00E94CE1363
:101A100081111BC060E2C62ED12C780109C08091D3
:101A2000F100D7018D937D01B1E0CB1AD10869F0A7
:101A30008091E80085FDF3CF8091E8008B7780935B
:101A4000E8000E94CE13882399F391E001C090E052
:101A50008091E8008B778093E800992309F415CEF4
:101A60002981822F90E0FC013197E331F10508F0E4
:101A70004EC1EE56FF4F0C9412231A828CE0B2C076
:101A80008A81823009F462C150F4813009F03FC18B
:101A90000E94AE149B838C837D836E833AC1833016
:101AA00041F0843009F033C11B821C821D821E82EA
:101AB00030C14B81D80180E090E0242F30E0B901A3
:101AC000680F791F6830710508F023C1E42FE80F13
:101AD000F0E0EE0FFF1FE257FE4F50816181139639
:101AE0006C93139714965C931497019612968E300C
:101AF000910529F70EC18A81823019F0853051F0A5
:101B000006C16B817C818D819E810E9418230E9479
:101B1000081CFFC08091530280FF03C00E94DC1E9E
:101B2000F8C00E94E91EF5C04C816B818A810E9439
:101B3000BF1D9D8312C12D813E813227232732276D
:101B40004C816B818A810E94531DE3C00E947A1DE3
:101B5000E0C08A81813009F0DAC02830F1F0293004
:101B6000B9F18B81813019F0823071F0D2C08C8153
:101B7000E3E08E9FC00111246FEF70E00E94C82245
:101B8000862F0E94C21EC5C08C81811103C00E9495
:101B9000971EBFC00E94AD1EBCC08B81813049F032
:101BA000823009F0B6C080915302869581708C8393
:101BB000B0C080915302869586958695FFEF8F9FE2
:101BC000C001112463E070E00E94C8226C83A1C0B0
:101BD000809153020E94911E9CC080E151C081E01F
:101BE0008A8388E98B8395C0EA80FB80FE24EF24FA
:101BF000FE24AC80B12C6801C70188599D4F960125
:101C0000201B310B2A153B0508F083C028E9E2169A
:101C100021E0F20630F40E946622D60114968C93DD
:101C200002C0F6011482FFEFEF1AFF0A2FEFC21A6B
:101C3000D20AE2CFEA80FB80FE24EF24FE24AC80AF
:101C4000B12C6801C70188599D4F9601201B310BAB
:101C50002A153B0508F05DC0A8E9EA16A1E0FA06DE
:101C600020F4F60164810E948422FFEFEF1AFF0A3C
:101C70002FEFC21AD20AE6CF0E94431D4AC084E069
:101C80008A8347C0EA80FB80FE24EF24FE24AC80D8
:101C9000B12C6801C70188969601201B310B2A15CB
:101CA0003B05B8F5A0E4EA16A2E0FA0628F40E9483
:101CB0006622F601848303C0D60114961C92BFEFFE
:101CC000EB1AFB0AEFEFCE1ADE0AE4CFEA80FB80C4
:101CD000FE24EF24FE24AC80B12C6801C701889655
:101CE0009601201B310B2A153B0598F4F0E4EF1602
:101CF000F2E0FF0628F4D60114966C910E9484222B
:101D0000BFEFEB1AFB0AEFEFCE1ADE0AE7CF8FEF39
:101D1000898340E250E0B80182E00E940114B5CC12
:101D2000E9BCF9BC09B400FEFDCF8091D8008F7DDD
:101D30008093D8008091E00082608093E0008091E1
:101D4000E00081FDFCCF0E940F20A8CC87E290E04C
:101D50000E9466221B821C821D828E83DACF2B306A
:101D6000310508F070CDA5CD2B30310508F0B7CD89
:101D7000ECCD8091B10187FF11C08091E80082FD18
:101D800005C08091AF018111F8CF11C08091E800AA
:101D90008B770BC08091AF01882349F08091E800D8
:101DA00080FFF8CF8091E8008E778093E800089557
:101DB000982F973068F59093E900981739F0709153
:101DC000EC002091ED005091F00003C0242F762FFD
:101DD00050E021FD02C09F5FECCF3091EB003E7FD1
:101DE0003093EB003091ED003D7F3093ED0030916A
:101DF000EB0031603093EB007093EC002093ED002A
:101E00005093F0002091EE0027FDE5CF80E008958B
:101E10008F708093E90081E008952091B70130919F
:101E2000B8012617370748F06115710539F420917C
:101E3000E8002E772093E80001C0B901FC0120E002
:101E40006115710579F18091AF018823F1F1853039
:101E5000F1F18091E80083FD3CC08091E80082FDB3
:101E60002EC08091E80080FFEBCF2091F30080919D
:101E7000F20090E0922B6115710551F088309105C8
:101E800038F421912093F100615071090196F3CF4C
:101E900021E0089709F020E08091E8008E77809398
:101EA000E800CECF2111CFCF0AC08091AF018823A7
:101EB00061F0853061F08091E80083FD0AC0809177
:101EC000E80082FFF2CF80E0089582E0089583E089
:101ED000089581E008958091A4010895AAE2B0E0F8
:101EE000E4E7FFE00C944823E1EBF1E089EB91E0BB
:101EF0002091F10021938E179F07D1F78091B201B5
:101F0000833009F463C030F4813071F0823009F419
:101F10009DC0B4C08A3009F489C08B3009F46EC00A
:101F2000893009F0ABC020C08091B101813A09F03D
:101F3000A5C08091E800877F8093E8008091B5017B
:101F40009091B601892B21F468E085EA91E003C005
:101F500060E080E090E070E00E940D0F8091E8006A
:101F60008B778093E8008AC08091B101813209F0BB
:101F700085C08091B5019091B601009719F0029744
:101F800009F07CC08091E800877F8093E800809111
:101F9000E80082FD05C08091AF018111F8CF6EC0CD
:101FA0002091F3008091F20090E0922B029731F49F
:101FB0008091F100813011F0863021F48091F100A0
:101FC0008093A4018091E8008B7754C08091B10187
:101FD000813A09F053C08091B5019091B601892BE7
:101FE00009F04CC08091E800877F8093E8008091E1
:101FF000E80080FFFCCF80910A0137C08091B101D9
:102000008132E1F58091B5019091B601892BB1F54E
:102010008091E800877F8093E8000E94B90E80914C
:10202000B30180930A010E940F2028C08091B10162
:10203000813221F58091E800877F8093E8000E943B
:10204000B90E8091B4018093A30118C08091B101B1
:10205000813AA1F48091E800877F8093E800809125
:10206000E80080FFFCCF8091A3018093F100809174
:10207000E8008E778093E8000E94B90E8091E80016
:1020800083FFDFC18091B1019091B201492F50E0EF
:102090004A30510508F0D5C1FA01EB55FF4F0C94B9
:1020A0001223803821F0823809F0CBC108C080911A
:1020B000AD019091AE01992389F082600FC08091AB
:1020C000B5018F70873008F0BCC18093E900809122
:1020D000EB0085FB882780F91092E9009091E800D9
:1020E000977F9093E8008093F1001092F10070C107
:1020F000282F2D7F09F0A5C1882319F0823061F0C7
:10210000A0C18091B301813009F09BC1933009F0E7
:1021100080E08093AE012EC08091B30181112AC06E
:102120008091B5018F702FEF280F263008F089C1FC
:102130008093E9002091EB0020FF1CC0933021F434
:102140008091EB00806214C09091EB0090619093BD
:10215000EB0021E030E0A90102C0440F551F8A9531
:10216000E2F74093EA001092EA008091EB00886069
:102170008093EB001092E9008091E800877F8093C4
:10218000E8000E94B90E5DC181115BC11091B301DD
:102190001F778091E3008078812B8093E30080910A
:1021A000E800877F8093E8000E94B90E8091E800E4
:1021B00080FFFCCF8091E30080688093E3001111E1
:1021C00002C082E001C083E08093AF013AC1805831
:1021D000823008F036C12091B3013091B4012C3D1A
:1021E00053E0350779F583E08A838AE289834FB724
:1021F000F894DE01139620E03EE051E2E32FF0E098
:1022000050935700E49120FF03C0E295EF703F5FC9
:10221000EF708E2F90E0EA3010F0C79601C0C096A4
:102220008D939D932F5F243149F74FBF8091E80034
:10223000877F8093E8006AE270E0CE0101960E94F9
:102240000D0FB4C08091B5019091B601432F552771
:1022500043305105A9F068F44130510509F400C13B
:102260004230510509F0EDC08BE590E0EAE2F3E081
:102270004BC04132510529F14232510589F1E1C08B
:10228000C901992781309105A1F058F0029709F012
:10229000D8C0E7E9F3E0E4918E2F90E0E7E9F3E0BE
:1022A00030C0E1EBF3E0E4918E2F90E0E1EBF3E05E
:1022B00028C0E3EAF3E0E4918E2F90E0E3EAF3E054
:1022C00020C08330910508F0BCC0880F991FFC0125
:1022D000EA5DFE4F0190F081E02D89E090E014C0AE
:1022E0008330910508F0ADC0FC01EE0FFF1FE05EEA
:1022F000FE4F0190F081E02DDC01A35EBE4F8C917A
:1023000090E0009709F49DC02091E800277F20937A
:10231000E8002091B7013091B8012817390708F477
:10232000C90140E0009789F12091AF01222309F40F
:102330003DC02530D9F12091E80023FD37C0209120
:10234000E80022FD2FC02091E80020FFEBCF409154
:10235000F3002091F20030E0342B009759F0283040
:10236000310540F444914093F100319601972F5F7D
:102370003F4FF3CF41E02830310509F040E0209194
:10238000E8002E772093E800CDCF4111CDCF0AC0D1
:102390008091AF01882351F0853041F08091E800B1
:1023A00083FD04C08091E80082FFF2CF8091E800B5
:1023B0008B778093E80045C0803809F042C0809157
:1023C000E800877F8093E8008091B0018093F1005E
:1023D0008091E8008E77D3CE811133C08091B30114
:1023E0009091B4019927029764F58091E800877F66
:1023F0008093E8001091B3011093B0010E94B90ED0
:10240000111106C08091E30087FD02C081E001C088
:1024100084E08093AF0142E061EC81E00E94D80E3D
:1024200042E261EC84E00E94D80E42E261EC82E07C
:102430000E94D80E42E260EC83E00E94D80E8091A8
:10244000AF018091E80083FF10C08091E800877F92
:102450008093E8008091EB0080628093EB0005C0E0
:1024600082E190E0E5E8F3E04FCFAA96E3E00C9438
:1024700064231F920F920FB60F9211242F933F9354
:102480004F935F936F937F938F939F93AF93BF937C
:10249000CF93DF93EF93FF93C091E900CF708091CA
:1024A000EC00D82FD17080FDD0E81092E900809127
:1024B000F000877F8093F00078940E946E0F109256
:1024C000E9008091F00088608093F000CD2BCF7000
:1024D000C093E900FF91EF91DF91CF91BF91AF9150
:1024E0009F918F917F916F915F914F913F912F912C
:1024F0000F900FBE0F901F901895E8EDF0E08081CF
:102500008E7F80831092E2001092DA001092E10038
:10251000A0EEB0E08C9181608C9380818F77808376
:1025200019BCA7EDB0E08C918E7F8C9380818F7E5B
:1025300080831092A2010895A0E0B0E0E2EAF2E107
:102540000C944323C8EDD0E088818F7E8883E7ED2B
:10255000F0E080818160808384E082BF81E08093AD
:10256000A20188818E7F888302EE10E0F80110823C
:102570001092DA0081EEC82ED12CF60110828881EB
:102580008F77888388818068888388818F7D88831E
:1025900019BC1092AF011092B0011092AE011092CE
:1025A000AD0190EEE92EF12CF70180818B7F8083C5
:1025B00088818160888342E060E080E00E94D80EDC
:1025C000F60180818E7F8083F80180818160808325
:1025D000808188608083F70180818E7F80838881FD
:1025E00080618883CDB7DEB7E8E00C945F231F924B
:1025F0000F920FB60F9211242F933F934F935F9337
:102600006F937F938F939F93AF93BF93EF93FF93BA
:102610008091E10082FF09C08091E20082FF05C045
:102620008091E1008B7F8093E1008091DA0080FF50
:102630002AC08091D80080FF26C08091DA008E7F6A
:102640008093DA008091D90080FF18C080E189BDB5
:1026500082E189BD09B400FEFDCF81E08093AF0126
:102660008091A20181110FC00E947D120E949C12D4
:102670008091E20084608093E20005C019BC109252
:10268000AF011092A2018091E10080FF17C08091FC
:10269000E20080FF13C08091E2008E7F8093E20011
:1026A0008091E20080618093E2008091D800806296
:1026B0008093D80019BC85E08093AF018091E10040
:1026C00084FF30C08091E20084FF2CC080E189BD8E
:1026D00082E189BD09B400FEFDCF8091D8008F7DD5
:1026E0008093D8008091E1008F7E8093E1008091FB
:1026F000E2008F7E8093E2008091E200816080930F
:10270000E2008091B001882311F084E007C080913D
:10271000E30087FD02C081E001C083E08093AF0148
:102720008091AF018091E10083FF27C08091E2009A
:1027300083FF23C08091E100877F8093E10082E0E6
:102740008093AF011092B0018091E1008E7F809361
:10275000E1008091E2008E7F8093E2008091E200B0
:1027600080618093E20042E060E080E00E94D80E49
:102770008091F00088608093F000FF91EF91BF910D
:10278000AF919F918F917F916F915F914F913F9109
:102790002F910F900FBE0F901F9018952091E4007D
:1027A0003091E50095E64091EC00842F817040FF68
:1027B00023C08091E80080FD1DC08091AF01882377
:1027C00099F0853099F08091EB0085FD11C0409122
:1027D000E4005091E5002417350729F3915011F0DA
:1027E0009A01E1CF84E0089582E0089583E008959E
:1027F00081E0089580E008954091E80042FFDDCF38
:1028000008950F931F93CF93DF938B01EA0190916B
:10281000AF01943079F58F708093E9008FEF90913C
:10282000E800815095FD06C095ED9A95F1F70000FE
:102830008111F5CF8091E80085FF1CC00E94CE1366
:10284000882361F08091E8008E778093E80012C0C1
:10285000F80181918F018093F1002197209791F3E6
:102860008091E80085FDF4CF8091E8008E77809319
:10287000E800E4CFDF91CF911F910F91089543E0DD
:1028800050E0BC0184E00E940114089546E050E04D
:10289000BC0184E00E940114089540E250E0BC01B4
:1028A00084E00E9401140895CF93DF93EC0148E087
:1028B00050E0BC0181E00E94011488E0FE01A5EA1D
:1028C000B1E001900D928A95E1F7DF91CF910895E3
:1028D00087E797E790930108809300089AE088E1E2
:1028E0000FB6F894A895809360000FBE9093600097
:1028F000FFCF78941F920F920FB60F9211248F93EF
:102900009F93AF93BF9380919E0190919F01A0915F
:10291000A001B091A1010196A11DB11D80939E015E
:1029200090939F01A093A001B093A101BF91AF919B
:102930009F918F910F900FBE0F901F9018959C0143
:102940004FB7F89480919E0190919F01A091A001B2
:10295000B091A1014FBF821B930B08952FB7F8943C
:1029600060919E0170919F018091A0019091A101C1
:102970002FBF08952FB7F89480919E0190919F01E9
:10298000A091A001B091A1012FBF089580E008950A
:1029900090916D0292FF10C041E0282F24712430E5
:1029A00009F040E031E0282F2871283009F030E0AC
:1029B000431711F02CE0822793FF10C041E0282F2D
:1029C0002471243109F040E031E0282F28712831AA
:1029D00009F030E0431711F02CE0822730916E02AD
:1029E00030FF10C051E0282F2171213009F050E054
:1029F00041E0282F2871283009F040E0541711F0E9
:102A000029E0822731FF10C041E0282F21712131B8
:102A100009F040E031E0282F2871283109F030E03A
:102A2000431711F029E0822794FD877E08958238AC
:102A3000910569F1B0F48133910509F475C048F44A
:102A40008932910509F467C08A32910509F471C091
:102A500008958533910509F459C089339105B9F07A
:102A60000895833E910589F138F4803E9105D1F0B7
:102A7000823E910529F10895863E9105C9F1873E70
:102A80009105D9F1843E910509F06CC027C02091D1
:102A90006D0220FD57C021FD55C020916E0223FD1F
:102AA0005BC0089580916D0280FD48C080916E02E8
:102AB00080FF48C080916D0284FD46C083EE51C006
:102AC00080916D0282FF3CC0F5CF80916D0282FD46
:102AD00037C080916E0280FD35C0ECCF80916E02D0
:102AE00081FF36C080916D0284FD2EC087EE39C013
:102AF00080916D0283FF2AC0F5CF80916D0283FD26
:102B000025C080916E0281FD23C0ECCF80916D02C3
:102B100085FD22C01FC080916D0285FD1BC0809184
:102B20006E0283FF19C00AC080916D0286FD16C037
:102B300017C080916D0286FD13C010C089E311C0DB
:102B400082EE0FC080EE0DC080E00BC086EE09C0A3
:102B500084EE07C085E305C089E203C08AE201C0B4
:102B600081E390E00895909125028091FC01892BEA
:102B70009091FB019923E1F0892B90910A0199230F
:102B800041F090916D0297FF04C09EE125E332E091
:102B900003C096E02DE232E0F90120E0915028F0E8
:102BA00031913323D9F32F5FF9CF21111092FB011B
:102BB00008952091F9019091C00157E02917A9F0DB
:102BC00030E0529FF001539FF00D1124EF53FE4F60
:102BD0007181761306C07081781303C075817413F8
:102BE00006C02F5F3F4F2770E9CF80E0089581E056
:102BF0000895F894E82FE295EF70F0E031A1282FC6
:102C00002F7081E090E001C0880F2A95EAF7982F95
:102C10009095932391A392A1892B82A378940895F0
:102C2000A0E1B0E0E6E1F6E10C943D23AE014F5F98
:102C30005F4F7A0180E1FA0111928A95E9F70CE081
:102C400011E06A0194E1692E91E0792E8824839441
:102C5000912CF80180818F3F09F447C0F894E82F48
:102C6000E295EF70F0E021A18F70A40102C0440F43
:102C7000551F8A95E2F7CA01922F982B91A392A132
:102C80008095892382A3789400C0E4E1F1E021E0FB
:102C900030E0A12CB12C41914F3F89F0A42FA29597
:102CA000AF70B0E090968C9190E04F7002C0959517
:102CB00087954A95E2F780FD02C0C90102C080E015
:102CC00090E0A82AB92A220F331F51E0ED31F50711
:102CD00011F7F80180818F3F11F00E94F915F0EA99
:102CE000FA95F1F7F601B182A0820F5F1F4FF2E073
:102CF000CF0ED11C6016710609F0ABCF40E150E059
:102D0000B7018AE691E00E947023892B91F080E15F
:102D1000F701AAE6B1E001900D928A95E1F781E012
:102D200080932A020E94BA14909329028093280269
:102D30000CC080912A02882341F080912802909152
:102D400029020E949F14059710F480E018C040E10A
:102D500050E06AE671E08EE891E00E947023892BD2
:102D600059F080E1EAE6F1E0AEE8B1E001900D92C1
:102D70008A95E1F781E001C080E010922A02609616
:102D8000EEE00C945923783048F4693038F48430FC
:102D900028F4462F672F0E94BF1D089580E090E021
:102DA00008951F93CF93DF930E941715EC01C1156F
:102DB00080E5D807E8F5C11590E4D90708F0A8C068
:102DC000C03ED10530F5CD3CD10508F094C0C83ADD
:102DD000D10578F4C53AD10508F083C0C130D105DA
:102DE00009F47CC008F4F2C0C430D10508F0F1C089
:102DF000EDC0C33CD10508F0E9C0C85AD0E0CC0F03
:102E0000DD1FC15DDE4F0990D881C02DCE019464D5
:102E1000E1C0C11580E2D80708F0CBC0C11591E030
:102E2000D90708F06BC0C83ED10508F4D2C0CEC0A7
:102E3000C03682E5D80728F5C03492E5D90708F0F6
:102E400079C0C03282E5D80708F06CC0C11592E5A0
:102E5000D90708F481C04C2F4695469580E2489FDB
:102E6000A0011124C37021E030E0C90102C0880F25
:102E7000991FCA95E2F7EA01C82BD92BCE019D68AC
:102E8000A9C0C03A82E5D807B8F48C2F8F71C0383A
:102E900092E5D90708F07BC08695869590E2899FD8
:102EA00090011124C37081E090E002C0880F991F47
:102EB000CA95E2F79A6868C0C03C82E5D80708F472
:102EC0006DC0C03E92E5D90708F080C0CF71DD2704
:102ED000DC2FCC27CE01806F906A7CC081E090E02F
:102EE00079C0C55AD0E0C45DDE4F8881C82FD0E0DC
:102EF000CE0190646FC0CE0190656CC08D2F0E9492
:102F0000C814182FCE0199270E9417151F715CC095
:102F1000CE0199270E941715CC27DF70D06A8C2B21
:102F20009D2B58C0CF71D0E0DC2FCC27CE01816F14
:102F3000906A50C08C2F8F718695869590E2899FFC
:102F400090011124C37081E090E002C0880F991FA6
:102F5000CA95E2F79C6818C08C2F8F710E94C81424
:102F600095E0D695C7959A95E1F7CF70D0E0DC2F24
:102F7000CC27282F30E084FF05C084E0220F331FC8
:102F80008A95E1F7D069CE01822B932B23C090E084
:102F9000D82FCC27CE01846F906A1CC08C2F8F71E4
:102FA0000E94C8148F7190E0D82FCC27CE01906278
:102FB00011C08D2F8F710E94C814182FCE01992730
:102FC0000E9417151F719062912B04C080E090E061
:102FD00001C0CE01DF91CF911F910895A6E0B0E02E
:102FE000E4EFF7E10C9447230E94BA148C0180911E
:102FF0002602909127020817190781F019821A8278
:103000000E94BA14682F49815A81792F80E090E09C
:103010000E94950310932702009326022696E4E06F
:103020000C94632380959091250289238093250237
:10303000089580910A01882351F180916D0287FFE4
:1030400026C00E94B3158093340240E250E06DEF39
:1030500071E083E392E00E947023892BD9F180E232
:10306000E3E3F2E0ADEFB1E001900D928A95E1F774
:10307000E0916902F0916A02309761F186E08093F5
:1030800033020480F581E02D83E392E022C00E94A8
:10309000B31580932B0248E050E06DE172E08BE2C3
:1030A00092E00E947023892BA9F088E0EBE2F2E025
:1030B000ADE1B2E001900D928A95E1F7E0916902ED
:1030C000F0916A02309731F00280F381E02D8BE2BB
:1030D00092E0099508959091FA0180958923809353
:1030E000FA01282F277069F4981759F090916E0211
:1030F00092FF07C08695869586950E94D01F1092F4
:10310000FA01089590916E0292FB222720F9281768
:1031100079F080FB92F990936E0260916D0270914C
:103120006E0284E090E00E94A22282E00E946B186E
:1031300008958091F9019091C001891719F08F5F6E
:103140008770FBCF0895CF93DF938091BF01829565
:103150008F7009F04EC08091BE01882309F449C0E8
:103160008091F9014091C0015091BA016091B9017B
:10317000C091BB01D091BC0177E08417D1F190E000
:10318000789FF001799FF00D1124DF01AF53BE4FFE
:1031900014962C911497222349F111962C91119792
:1031A000251324C02C91261321C015962C91159718
:1031B00021111CC012962D913C9113972C1B3D0B95
:1031C000283C310598F48091BF018F708061809315
:1031D000BF01E953FE4F80818F708061808389EB4E
:1031E00091E00E9425040E94991803C001968770FF
:1031F000C4CFDF91CF910895A4E1B0E0E2E0F9E11E
:103200000C943F238C0186E0F801DE011F960190AB
:103210000D928A95E1F7F8018481E58099EB892E7A
:1032200091E0992E9091BD01911120C0882309F45D
:1032300063C1EE2009F442C0C8010E94EC1FF82EC1
:103240008823E1F187E0F801D40101900D928A957D
:10325000E1F78091BD01813031F48091B901909105
:10326000BA010E94571F0E94A31848C1F801D080DC
:10327000C180A280B380F090BE012091BB0130914B
:10328000BC01FF2009F4E7C0A501421B530B483CD9
:10329000510508F09DC0882309F430C18091BF0119
:1032A000282F207F9091BA01222361F09C1509F408
:1032B00060C0C8010E94EC1F811163C0C8010E9458
:1032C00025041AC19C1113C09091B9019D110FC022
:1032D000E1100DC08F7080618093BF0189EB91E098
:1032E0000E9425048091BF01F801868303C1E1108B
:1032F0003AC040E06C2D8D2D0E94D91540E06C2D18
:103300008D2D0E94D915E82E8111F4C0DF86C88A60
:103310008F8598890E94571F292F22952F7024305E
:1033200020F49F70223028F009C02A50223080F00B
:1033300014C0992349F0811107C013C0992321F0CB
:10334000F8019681907F69F0805E883030F409C082
:10335000803F38F0815F833020F0C8010E9425044F
:10336000EF2CFE2CCBC08091BF0181608093BF0108
:10337000C1C09091B9019D119CCFE1109ACFF80185
:1033800098C0EE2009F49ACF2091BF01822F829538
:103390008F7090E002978CF08091B9019091BA0102
:1033A00099878887BB86AA868091BD018C871D86F8
:1033B0002E87CE0108960E94250487E0F801A9EB2C
:1033C000B1E001900D928A95E1F70E94A31894C094
:1033D0009091BF01292F207F51F489EB91E00E9449
:1033E000250487E0F40111928A95E9F783C08823C8
:1033F00009F484C08091BA018C110CC08091B9018C
:103400008D1108C0E11006C0F8019683C8010E9422
:1034100025046AC0C8010E94EC1F882309F44ECF1E
:10342000EE2009F44BCF2091BF01822F82958F703F
:1034300090E0029714F28091B9019091BA019A83B9
:103440008983BC82AB828091BD018D831E822F83D4
:10345000CE010196B0CFA21AB30AF8ECAF16B104B0
:1034600008F042C0882309F447C0FE2CEE2009F47E
:1034700025CF8091BA018C1129C08091B9018D119D
:1034800025C09091BF0190FD18C0892F82958F7043
:10349000282F30E02115310581F0F80196832F3077
:1034A000310541F08F5F982F9295907F86818F70C4
:1034B000892B8683C8010E94250487E0F801A9EBC7
:1034C000B1E001900D928A95E1F718C0C8010E9401
:1034D000EC1F811172CF8091BF0181608093BF0189
:1034E000C8010E9425040AC087E0F40111928A9560
:1034F000E9F704C0F12C02C0FF24F3948F2D6496E9
:10350000ECE00C945B2390917B0121E030E0F90129
:1035100001C0EE0F8A95EAF7D90102C0AA0FBB1FBE
:103520006A95E2F7BD016E2B01C0220F4A95EAF7BA
:10353000892F8623681303C0892F822B03C020950F
:10354000822F89230E94CD1F0895A0E0B0E0EBEA0E
:10355000FAE10C943F238C018091860090918700C2
:103560006CE070E00E94C8226017710730F0C8015B
:1035700069E070E00E94C82260C08091860090914E
:103580008700E0908600F0908700E0918600F0913F
:103590008700C6E0D0E0BE010E94C82220E030E0F3
:1035A000060F171F211D311D4801590185E0880CA8
:1035B000991CAA1CBB1C8A95D1F7C701BE010E94A9
:1035C000C8226F01E12CF12CA7019601260F371FAD
:1035D000411D511DC501B4010E94F02269017A010B
:1035E000E0918600F0918700CA01B9010E94B822DB
:1035F0009B01AC01DF010E942E239B01AC01C7019E
:10360000B6010E94B822DC01CB012FE0B695A79548
:10361000979587952A95D1F700918600109187009C
:1036200020E030E0081719072A073B0728F46091CB
:10363000860070918700CB01BC01CB01CDB7DEB70E
:10364000ECE00C945B231F920F920FB60F921124A3
:103650008F939F93AF93BF9380916F02811113C09B
:1036600080919E0190919F01A091A001B091A10134
:103670004196A11DB11D80939E0190939F01A0933F
:10368000A001B093A101BF91AF919F918F910F9035
:103690000FBE0F901F90189590910A01992321F069
:1036A00090916D0297FD03C0EBE2F2E01DC0E82FA0
:1036B000E695E695E695EE31E0F4F0E0ED5CFD4F41
:1036C000877021E030E0A90102C0440F551F8A95A0
:1036D000E2F7CA0180959281892382830895319609
:1036E00052E0E133F50729F092818913F8CF128275
:1036F000F6CF089590910A019923D1F090916D022F
:1037000097FF16C0E82FE695E695E695EE3140F571
:10371000F0E0ED5CFD4F877021E030E0A90102C0D0
:10372000440F551F8A95E2F7CA019281892B16C072
:10373000ADE2B2E0EFEF90E02D91821789F0EF3F1C
:1037400019F4211101C0E92F9F5F9630A9F7EF3FCF
:1037500039F00E2E000CFF0BE55DFD4F82830895BE
:103760000895A3E0B0E0E7EBFBE10C94492320913E
:103770006B0230916C0228173907A1F090936C020C
:1037800080936B02E0916902F0916A02309751F0E8
:1037900024E029839B838A830084F185E02DCE0178
:1037A000019609952396E2E00C946523A3E0B0E02E
:1037B000ECEDFBE10C944923209167023091680203
:1037C00028173907A1F09093680280936702E0916F
:1037D0006902F0916A02309751F023E029839B83BC
:1037E0008A830084F185E02DCE0101960995239608
:1037F000E2E00C946523E0916902F0916A0230974F
:1038000029F00190F081E02D0995089580E0089558
:1038100087E290E00E9484220895CF93C82F8111FF
:1038200002C06FEF01C064E284E290E00E94842253
:10383000C11102C06FEF01C068E085E290E00E9414
:103840008422C11102C06FEF01C067E186E290E0FF
:103850000E948422CF91089584E290E00E94662223
:10386000843281F485E290E00E946622883051F42F
:1038700086E290E00E94662291E0873109F090E0B4
:10388000892F01C080E0817008950F931F93CF931B
:10389000DF93C42FD22FFC0185818823B1F04093A0
:1038A00066020E94BA14909365028093640280E2DB
:1038B0008C0F883008F068C0C77081E001C0880FA5
:1038C000CA95EAF70E9447205FC0809166024813BC
:1038D0003DC080916402909165020E949F14883CD3
:1038E0009105A0F510E21D0FCD17E9F080E28C0FD5
:1038F000883040F4C77081E001C0880FCA95EAF7AC
:103900000E944020183078F581E09D2F977001C00B
:10391000880F9A95EAF70E944720093351F560E530
:1039200070E089E329C0093319F460E570E002C052
:1039300060E070E0802F0E944E22183028F5D7708A
:1039400081E001C0880FDA95EAF70AC080E28C0FA7
:103950008830D0F4C77081E001C0880FCA95EAF7BB
:103960000E94402011C0093351F460E570E089E302
:1039700009C060E070E0802F0E944E22E0CF60E03E
:1039800070E0802F0E944E22DF91CF911F910F9106
:1039900008950E94BA1420916002211104C0209160
:1039A0006102222321F090935D0280935C022091BA
:1039B0006202211104C020916302222321F090931E
:1039C0005B0280935A02E0916902F0916A0230979B
:1039D00049F082E080935E020680F781E02D8EE55B
:1039E00092E0099508958091590280FD16C081FDED
:1039F00016C082FD18C080915802882391F0883249
:103A000090F428E0829FC001112468E270E00E94D7
:103A1000DC22862F672B29F007C082E0089584E01E
:103A2000089581E0089588E008958091590280FD0D
:103A300014C081FD14C082FD16C0809157028823F6
:103A400081F08E3180F420E5829FC00111246EE167
:103A500070E00E94DC22862F089584E1089588E2B8
:103A6000089588E0089580E50895282F35EB230315
:103A7000C001112497FF03C08058910902C08058EB
:103A80009F4F892F0895CF93DF93C8E6D2E060E07F
:103A9000CE010E9484222196C11584E0D807B9F78F
:103AA000DF91CF9108951F93CF93DF93962F8430AA
:103AB000E8F46830D8F44930C8F4632F122FC42FCB
:103AC000D0E0CC0FDD1F22E1929FC00DD11D11244B
:103AD00090E9899FC00DD11D1124CE0188960E94C6
:103AE0008422612FCE0189960E948422DF91CF919A
:103AF0001F910895A0E0B0E0E0E8FDE10C944123BF
:103B0000A12CE12CF12CB12C00E010E0C0E0D0E0C1
:103B10006701C00ED11EFE01EE0FFF1FEC0DFD1D53
:103B2000EB5CFB4F259134914C2F6B2D8A2D0E941D
:103B3000531D2196C930D10571F70E5E1F4FB39406
:103B400088E0B812E3CF80E9E80EF11CA39484E08A
:103B5000A812D9CFCDB7DEB7EAE00C945D2380E0A0
:103B60000E940D1C60E070E0CB010E94081C0E94C6
:103B70007A1D0E94431D81E00E940D1C08950F9341
:103B80001F93CF93DF93843008F56830F8F4493001
:103B9000E8F4C42FD0E0CC0FDD1F22E1629FC00DFE
:103BA000D11D112430E9839FC00DD11D1124CE01F8
:103BB00088960E94662290E0182F0027CE018996F1
:103BC0000E9466229801282BC90102C080E090E083
:103BD000DF91CF911F910F9108951F920F920FB611
:103BE0000F9211242F933F934F935F936F937F9383
:103BF0008F939F93AF93BF93EF93FF9380910B01AC
:103C000091E0980F823019F090930B014EC081E043
:103C100080930B018091550290915602019660EDC0
:103C200072E00E94C822909356028093550265E08C
:103C300070E00E94C82267FD6FE7809154028230D5
:103C400019F4603451F404C0813039F46F3729F429
:103C500080916F008E7F80936F00E62FF0E0EB5431
:103C6000FC4F2491A0918600B091870030E00E9423
:103C70001F232FEF30E040E050E00E94F022C90106
:103C800063E070E00E94C822809153028695869579
:103C90008695282F269FC001279F900D11240E94F2
:103CA000A51A9093890080938800FF91EF91BF91AE
:103CB000AF919F918F917F916F915F914F913F91C4
:103CC0002F910F900FBE0F901F901895843030F4F5
:103CD000811105C0909180009F7704C083E090918E
:103CE0008000906890938000A0918600B09187003A
:103CF000282F30E00E941F2323E030E040E050E016
:103D00000E94F022B42FA32F922F8827892F9A2F59
:103D1000AB2FBB270E94A51A90938900809388003F
:103D20000895682F86E090E00E9484220895809193
:103D3000530281FF11C08D7F809353020E94911E18
:103D400080916F008E7F80936F00809153028695E3
:103D5000869586950E94661E08958091530281FD86
:103D600010C08260809353020E94911E10925602EE
:103D7000109255021092540280916F0081608093DE
:103D80006F000895843008F083E09091530297709B
:103D9000282F220F220F220F922B90935302987FED
:103DA00021E009F420E09091530220FB90F99093D8
:103DB00053020E94661E08958091530280FF08C03E
:103DC0008E7F809353020E94911E80E00E94661EA7
:103DD00008958091530280FD13C081608093530247
:103DE000813019F489E080935302809153020E943C
:103DF000911E809153028695869586950E94661E37
:103E0000089586E090E00E9466228093530282FD2E
:103E100005C08DE1809353020E94911E8091530250
:103E2000282F26952695269530E02430310524F05C
:103E300087708861809353028091530280FF04C091
:103E400086958695869501C080E00E94661E08953D
:103E5000CF92DF92FF920F931F93CF93DF936C016A
:103E600000917B0180917A01082BC3E0D0E010E043
:103E7000C8010C2E02C0959587950A94E2F780FD43
